:1000000019C028C027C026C025C024C023C022C0D4
:1000100021C020C01FC01EC01DC01CC0A1C01AC06E
:1000200019C018C017C016C015C014C013C012C024
:1000300011C010C011241FBECFEFCDBFDFE3DEBF64
:100040002FE3A0E0BFE301C01D92AA30B207E1F7A1
:10005000DDD039C1D5CF9091010A9B7F9093010AE1
:100060009091000492FF0AC0811104C084E0809343
:100070000604089584E08093050408959FB7F894DA
:10008000811107C080911204877F809312049FBF63
:100090000895809112048860F8CF8FB7F89420916A
:1000A000063F3091073F4091083F5091093F98E04B
:1000B0009093840A90918E0A91FFFCCFE091A20A5E
:1000C000F091A30A90918D0A90FF08C0BF016627A6
:1000D000672B21F42E5F3F4F4F4F5F4F8FBFBF0104
:1000E00076956795CF01860F911DE62FE695E695EB
:1000F000762F72957F70E71BFF0B67FD3196E80F37
:10010000F91FA0E3B3E0C9D06E0F7F1F811D911DC1
:100110000895CF92DF92EF92FF92BFDF6B017C01D7
:1001200020E4C20E22E4D21E2FE0E21EF11C80E485
:10013000C81682E4D8068FE0E806F10430F4ADDF9B
:10014000C616D706E806F906D0F3A7DF6C157D05BD
:100150008E059F05D0F3FF90EF90DF90CF9008952C
:100160001F920F920FB60F9211242F933F934F932C
:100170005F936F938F939F93AF93BF938091023F51
:100180009091033FA091043FB091053F4091003F03
:100190005091013F9A01205D3C4F283E63E03607B5
:1001A00028F0285E33400196A11DB11D2093003F29
:1001B0003093013F8093023F9093033FA093043F0D
:1001C000B093053F8091063F9091073FA091083F73
:1001D000B091093F0196A11DB11D8093063F9093F8
:1001E000073FA093083FB093093F81E080938D0AB9
:1001F000BF91AF919F918F916F915F914F913F917F
:100200002F910F900FBE0F901F90189588ED90E0E2
:1002100084BF9093610083E5809302068EE0809313
:10022000050680E28093030680910006816080933A
:10023000000691E0909302029093030A8EEF809360
:10024000260A8093270A80E88093280A80932A0A46
:1002500080932C0A8093290A80932B0A80932D0A7D
:100260002BE02093000A2DEF31E02093AE0A30936B
:10027000AF0A90938C0A1092810A8093820A81E1DE
:100280008093800A789484E08093010481E0E3DE27
:1002900040DF80E0E0DE3DDFF9CF09D0A59F900D83
:1002A000B49F900DA49F800D911D11240895A29FCD
:1002B000B001B39FC001A39F01D0B29F700D811DFB
:0A02C0001124911D0895F894FFCF5A
:00000001FF
